:020000040000FA
:020000000528D1
:08000800CF2B031383129F01AB
:10001000831606309F003F308500860180308700C0
:1000200088018901803081000C108312013090001A
:100030008601870187160000871288018901053033
:10004000C100C001051C40143C230C3012230230B7
:10005000AC003D30AD007423C030122374230B1765
:100060008B179B230530A1008815C12388118914A3
:10007000C12389100915C1230911A10B3428C923F3
:10008000013012230230AC005F30AD007423C03069
:1000900012237423C92301301223C923C72301303B
:1000A00012230230AC008130AD007423C030122323
:1000B00074239B23C723A2010D3012232208A520FD
:1000C000A50080381223051C6A28851CC522051D41
:1000D000D3225E28C723013012233C301423023080
:1000E000AC008130AD002508A600261F7D28BF305A
:1000F000A6050230AC009230AD00A701AD0A03198D
:10010000AC0AA60B7E287F238A110A121423AD0A9B
:100110000319AC0AA70A04302702031D83283E30C6
:1001200014230D301223883012230230AC00A33088
:10013000AD0074239B23C723851D4E2805189C28DA
:10014000BD019B23851CBD0AB328AF3EAD00003026
:100150000318013EAC007F238A110A1208000734FD
:100160000C3447344C34050E0339033AA4000230F2
:1001700022020318C22803302402031DC228C72309
:10018000A8239C280C301223883012230230AC00A4
:10019000AB30AD007423C030122374238815E122E4
:1001A000870102302202031DD6280717BA01BB01BE
:1001B000BC012408031DF528B401B5018C21B70149
:1001C0009D21BC21E7213E187A29851D7A29B70A8D
:1001D000023022020230031810303702031DE028DB
:1001E0001922BF080319DE287A2901302402031DD1
:1001F0001929B701B401B5018C219D211922BF082D
:100200000319FC28B401B5018C21BC21E7213E185B
:100210007A29851D7A291922BF0803190429B70AEA
:10022000023022020230031810303702031DFA2870
:100230007A2902302402031D5D29B801B401B501F9
:100240003808B7008C219D211922BF08031D3229CF
:10025000B70A0230220202300318103037020319A5
:10026000B7012229B401B5013808B7008C21BC219F
:10027000E7213E187A29851D7A291922BF08031D16
:100280004B29B70A0230220202300318103037021D
:100290000319B7013629B80A0230220202300318C6
:1002A00010303802031D1E297A2901340234043427
:1002B000083400340F3405340A34B401B5018C21FC
:1002C0000130AC005530AD007F238A110A12AD0A0F
:1002D0000319AC0AB7009D21BC21E7213E187A29F9
:1002E000851D7A290A303702031D64291922BF08A7
:1002F00003195F29BC08031980290915A82382293D
:100300008914A023860187018716000087128811AF
:100310000518882989016B28C23012233408282245
:10032000350828223508860000008716000087124D
:100330000F308605340E86040800C93012233708B2
:100340002822023022020318AA2907133708031DA6
:100350000717AF29F03086053708860400003908F2
:1003600087040000000007160000000000000712CC
:100370000000F03087050800023022020318C72968
:10038000390887040000B601871BB60AE029031369
:1003900083160F3086008312340E860039088704D6
:1003A00002302202031DD529071306080F39B600B3
:1003B00002302202031DDD290717831686018312EE
:1003C000F0308705CE301223360828220800BE01FF
:1003D000C0080319FD294108CA238518F229C10361
:1003E0000319C10A41080519F829013E831CC100FF
:1003F00087301223410832221423360837020319AA
:10040000182ABB0A0319BA0A3C148C3012233A0882
:1004100028223B082822BD080319182A091583231E
:100420008519142A3E14182A0519102A0911C72300
:100430000800BF0143083502031D242A4208340284
:10044000031D242A3F14272AB50A0319B40A0800F9
:10045000C600460E0F39322214230F3046053222D1
:1004600014230800C7000A3C03193A2A031C3A2A3D
:1004700030303B2A37304707080053347434613436
:10048000743469346334523461346D3443346834C1
:10049000653463346B34653472340034203428346A
:1004A0003134203462346934743420342F342034AD
:1004B00034342034623469347434293400342034C0
:1004C0002034203420347634653472342E34313480
:1004D0002E3430343234203420342034203400346C
:1004E000203420346234793420346D342E3479341D
:1004F00061346D3461346D346F3474346F3420344E
:10050000003454347934703465343F345F342034EB
:1005100032343134303432342034343430343434BE
:100520003434003420342034203420342034203437
:1005300020343534313430343134203432343134B1
:100540003134343400345334743461347234743498
:100550003F345F3400342034453472343A3430341C
:10056000303430343034003441343A3420342034A0
:1005700020342034203457343A342034203420348A
:1005800052343A342034203400341E30C2238518CB
:10059000D22A95239630C223A203220A031DD22A0F
:1005A0000330A20008001E30C2230519E02A95235B
:1005B0009630C223A20A04302202031DE02AA201BF
:1005C00008000330AC000630AD002208C400C408A7
:1005D0000319F32A0330C500AD0A0319AC0AC50B91
:1005E000EC2AC403E72A7F238A110A12B900AD0A54
:1005F0000319AC0A7F238A110A12C200AD0A03193B
:10060000AC0A7F238A110A12C300080001340334A4
:10061000FF3402340F34FF3404340034FF34083420
:100620000334FF340811162B0815000088101C2312
:10063000200E1C2326230800A0000F308805F03070
:100640002005880408140000081008008316F03004
:100650008804831208110000881408140808081080
:10066000A000081408080810A01B2D2B8810831662
:10067000F03088068312080088100000081100007E
:1006800008100F30C22330301C230530C223303015
:100690001C23B52330301C23B52320301C23B52365
:1006A000283012230830122301301223063012237F
:1006B00008008316F030880483120815000088149F
:1006C000081408080810F039A000A00E0814080843
:1006D0000810F039A004A00E88108316F0308806A8
:1006E0008312B523200808007F238A110A12AD0A5D
:1006F0000319AC0A003E031908001423742B2C08BC
:100700008A002D088200DA30AE00AD30AF00FA303A
:10071000AD2BDA30AE00AD30AF004630AD2BE73058
:10072000AE001730AF004630AD2BED30AE00573085
:10073000AF004630AD2B8F231E30C2239523080017
:100740000430B30095231E30C223B30BA22B080044
:1007500089234630C2238323080083160C14831296
:10076000C22383160C10831208006330B000B82B2C
:10077000B00BB72B08000A30B100B523B10BBD2B6D
:1007800008006430B200BB23B20BC32B0800053055
:10079000CA2B0F30B300C123B30BCB2B0800F000E2
:1007A0000308F100831203130C1CDD2B2E088F00AD
:1007B0002F088E00013089060C1071088300F00E9E
:0407C000700E0900AE
:02400E00323F3F
:1042000043006F0070007900720069006700680069
:1042100074002000280043002900200032003000F4
:104220003100300020006200790020004D002E0097
:10423000590061006D0061006D006F0074006F0037
:00000001FF
